:100000000BC6000026C6000024C600000C94C029C0
:1000100020C600001EC600001CC600001AC6000054
:1000200018C6000016C600000C948A260C9472278D
:100030000C9483100EC600000CC600000AC6000017
:1000400008C6000006C6000004C6000002C6000084
:1000500000C600000C946626FCC50000FAC500002E
:10006000F8C50000F6C50000F4C50000F2C50000A8
:10007000F0C50000EEC50000ECC50000EAC50000B8
:10008000E8C50000E6C50000E4C50000E2C50000C8
:10009000E0C50000DEC50000DCC50000DAC50000D8
:1000A000D8C50000D6C50000D4C5000005010980F0
:1000B000A101850319012AB700150126B700950192
:1000C00075108100C0050C0901A101850419012AE0
:1000D000A002150126A002950175108100C00660DE
:1000E000FF0961A1010962150026FF00952075082E
:1000F00081020963150026FF00952075089102C052
:1001000005010906A101050719E029E715002501E8
:10011000950875018102950175088101050719008F
:1001200029FF150026FF00950675088100050819AE
:1001300001290515002501950575019102950175A7
:10014000039101C000AF00AE0000000000003E5B64
:100150004F5B3E003E6B4F6B3E001C3E7C3E1C00E6
:10016000183C7E3C18001C577D571C001C5E7F5EAF
:100170001C0000183C180000FFE7C3E7FF00001850
:1001800024180000FFE7DBE7FF0030483A060E00C6
:10019000262979292600407F05050700407F05258F
:1001A0003F005A3CE73C5A007F3E1C1C0800081CDC
:1001B0001C3E7F0014227F2214005F5F005F5F00FF
:1001C00006097F017F00006689956A0060606060B3
:1001D000600094A2FFA2940008047E04080010208E
:1001E0007E20100008082A1C0800081C2A080800A5
:1001F0001E10101010000C1E0C1E0C0030383E3863
:100200003000060E3E0E0600000000000000000058
:100210005F000000000700070000147F147F140037
:10022000242A7F2A120023130864620036495620CC
:100230005000000807030000001C2241000000419C
:10024000221C00002A1C7F1C2A0008083E08080007
:100250000080703000000808080808000000606096
:1002600000002010080402003E5149453E000042B3
:100270007F4000007249494946002141494D330001
:100280001814127F10002745454539003C4A49495A
:1002900031004121110907003649494936004649D4
:1002A00049291E0000001400000000403400000036
:1002B00000081422410014141414140000412214E4
:1002C00008000201590906003E415D594E007C12AA
:1002D00011127C007F49494936003E4141412200CC
:1002E0007F4141413E007F49494941007F09090959
:1002F00001003E41415173007F0808087F00004122
:100300007F4100002040413F01007F08142241004E
:100310007F40404040007F021C027F007F040810A5
:100320007F003E4141413E007F09090906003E41F0
:1003300051215E007F0919294600264949493200AA
:1003400003017F0103003F4040403F001F20402049
:100350001F003F4038403F0063140814630003044B
:10036000780403006159494D4300007F4141410039
:10037000020408102000004141417F0004020102F4
:1003800004004040404040000003070800002054A3
:10039000547840007F2844443800384444442800BE
:1003A000384444287F0038545454180000087E090B
:1003B000020018A4A49C78007F080404780000447C
:1003C0007D4000002040403D00007F102844000098
:1003D00000417F4000007C04780478007C0804041D
:1003E0007800384444443800FC18242418001824A9
:1003F0002418FC007C0804040800485454542400C9
:1004000004043F4424003C4040207C001C20402049
:100410001C003C4030403C004428102844004C90D4
:1004200090907C004464544C440000083641000025
:1004300000007700000000413608000002010204BD
:1004400002003C2623263C0003071F7FFFFFFEF827
:10045000F0C020F8FEFFFE79271F7FFFFFFEF8F0B7
:10046000C020F8FEFFFF7F3F3F7FFFFEF8F0C00097
:10047000000000FFFFFFFFFFFF0000000000000082
:10048000FF7F7F7FBFBFC0C0C0E0E0E0E0F0F0F0E2
:10049000F878787C3C3CFEFEFEFFFFFF0000000089
:1004A0000000000000008080BFBFDFDFEFEF00032F
:1004B000071F7FFFFFFFFEF8E0C0E0F8FEFFFFFF31
:1004C0007F1F07030000E0F0F0F0E0ECEEF7F370C0
:1004D00020007C7C7C7E007E7E7E7F7F7F00008093
:1004E000C0E07E5B4F5BFEC00000C000DCD7DEDEFC
:1004F000DED7DC00C00000000000000000000000AB
:10050000000000000000000000000000C1F3CFBFA9
:100510007FFFFFFCFBE7810000000080E3CF3FFF8F
:10052000FFFFFCFBE7810000000081E7FFFFFFFF0A
:100530003C0000FFFFFFFFFFFFF8F8FC7C7E7E3EE3
:10054000FEFFFFFFFFFFF7F7F7FBFB7D7D7DBEBEE4
:10055000BEDFDFE0E000FFFFFFFFFFFF00FCFC7CF1
:100560007E7E3E3E1F1F1F0FFFFFFFFFFFFF0000AD
:1005700000000081E7FFFFFFFFFFFFFFFFFFE781B4
:100580000000000000000F1F3F7F7F7F7F7F3F1E26
:100590000C001F1F1F3F003F3F3F7F7F7F00307BCE
:1005A0007F7830202030787F3B0003000F7F0F0FD3
:1005B0000F7F0F000300000000000000000000009B
:1005C000000000000000000060707C7F7F7F7F1FC4
:1005D0000601030F3F7F7F7E7C7C7E7F7F7F1F062F
:1005E00001070F3F7F7F7E7C7C7E7F7F3F0F030074
:1005F0000000007F7F7F7F7F7F0000000000000001
:100600007F7F7F7F7F7F7D7D3D3E1E1F1F1F0F0FE2
:100610000707070303007F7F7F7F7F7F7C7C7C7CD5
:100620007C7C7C7C7C7C7C007F7F7F7F7F7F00402C
:1006300070787E7F7F7F3F0F0301030F3F7F7F7FB7
:100640007E78704000000000000000000000000004
:10065000000000000000000000000000000000009A
:10066000000000000000000000000000000000008A
:10067000000000000000000000000000000000007A
:10068000000000000000000000000000000000006A
:10069000000000000000000000000000000000005A
:1006A0000000000000000000000000007E0F00D4E9
:1006B000FFFFFFC7000000780000000000000000FE
:1006C0002A2B2800000000000000000000000000AD
:1006D00000000029000000002C1E342021222434B8
:1006E0002627252E362D3738271E1F20212223248A
:1006F00025263333362E37381F0405060708090A26
:100700000B0C0D0E0F101112131415161718191AC1
:100710001B1C1D2F3130232D350405060708090A3F
:100720000B0C0D0E0F101112131415161718191AA1
:100730001B1C1D2F3130354C09025B00030100A04A
:100740003209040000010301010009211101000127
:100750002244000705810308000109040100020387
:100760000000000921110100012222000705820377
:100770002000010705030320000109040200010312
:100780000000000921110100012232000705840345
:100790002000011201000200000008653200000183
:1007A00000010203011C037600690061006C003A3D
:1007B00000660036003400630032006200330063DC
:1007C0000000001603480065006C006900780020F6
:1007D00000420065007400610000001403590075B8
:1007E000007300680061006B006F0062006F000022
:1007F000000403090435001E001F00200021002210
:100800000000002B0014001A00080015001700005B
:1008100000E00004001600070009000A000000E1E3
:10082000001D001B000600190005002F00457E2951
:1008300000E200E300477E437E2C004C00270026A8
:100840000025002400230000002A00130012000CE1
:100850000018001C000000340033000F000E000DD3
:10086000000B00000028003800370036001000118F
:100870000030004F00520051005000487E447E2C52
:100880000035001E001F0020002100220000002B68
:100890000014001A00090013000A000000E0000420
:1008A0000015001600170007000000E1001D001BE6
:1008B000000600190005002F00457E2900E200E334
:1008C00000477E437E2C004C002700260025002494
:1008D00000230000002A0033001C0018000F000D48
:1008E000000000340012000C00080011000B000092
:1008F00000280038003700360010000E0030004F8E
:1009000000520051005000487E447E2C0035001EED
:10091000001F0020002100220000002B00340036C0
:1009200000370013001C000000E000040012000863
:100930000018000C000000E100330014000D000E50
:10094000001B002F00457E2900E200E300477E43A4
:100950007E2C002A0027002600250024002300000A
:10096000004C000F00150006000A000900000038C6
:10097000001600110017000B000700000028001DE2
:100980000019001A001000050030004F00520051FD
:10099000005000487E447E2C0035021E021F0220BB
:1009A0000221022202000035021E021F0220022143
:1009B000022202000001003A003B003C003D003EE4
:1009C000000000390040004100420043004400267E
:1009D000020100010001000100010001000100010D
:1009E000002702260225022402230200000100271C
:1009F0000226022502240223020000310230022FC7
:100A0000022E022D023F00000001004D004A0001AD
:100A100000010045002702AE00A900AA00AB0001BA
:100A2000000100010000DA0281FFD9F1DB20A4A659
:100A30002EAF00A0C0D30000A1C8D30000AED58067
:100A4000A81F408D1420008081828384858687883A
:100A5000898A8B8C8D8E8F9091929394A0A1A2A362
:100A6000A4A5A6A7A8A9AAABACADAEAFB0B1B2B3CE
:100A7000B4C0C1C2C3C4C5C6C7C8C9CACBCCCDCE19
:100A8000CFD0D1D2D3D400202020200053434C4BD0
:100A9000002020202000434150530020202020200F
:100AA0002020004E554D4C4F434B00FD377A585A8D
:100AB000000004E6D6B446020021011600000074CE
:100AC0002FE5A3E002E301195D003D8889C6543695
:100AD000C3174FE4DFB5E4CD54789055FA8F966094
:100AE0005BDAEDD40E6D961DB3AC9B07994D5F4755
:100AF000239EA4B2691FAB764FA85C521872AEA4B5
:100B0000ABA06D9DFC6AA4FF912304F713CDCD5DCE
:100B1000157F264A187DE9FFB09A9ADF64676AA0BC
:100B20001D4C6A34C59875F918AAE7635023571409
:100B300025CD57DC780A62D56FDA52DDD77005AD66
:100B4000DF7DAEDD5177B48D3E3F8FABBD1C0B0F0B
:100B50002745965553A810A990DCE9DB9A87FA74CB
:100B6000CC7A98AC25802298043AC2D6E69A55AF42
:100B7000131DE129890CE1AA69CF6D6EE93F03528B
:100B8000AF39CC0EF3B878CF5A580520EED4A8AFC1
:100B900057B4703660CDA5FAD010EEDC59B8A46F0A
:100BA00092A0A9903423A281F76E06FD3C90476481
:100BB000337E4605BD9D7D7728A208CB21E0515D9F
:100BC000B423E9A106B594A802ACDCA7878F42A2A2
:100BD000BA3EA42D6950744575164C5F95B1B52B7E
:100BE000C7971100000000C4140987D7AD3A070069
:100BF00001B502E4050000FF1144ACB1C467FB027B
:100C00000000000004595A0102E2600103E2000101
:100C100002E2600103E2000011241FBECFEFDAE020
:100C2000DEBFCDBF11E0A0E0B1E0E0ECF7E502C02F
:100C300005900D92A23EB107D9F725E0A2EEB1E0F2
:100C400001C01D92A032B207E1F70E940C200C9463
:100C5000A32BD6C99C01FB019A9581159F4120F5D4
:100C6000832F8170B32FB270AA27732F74706627F9
:100C7000532F5870442734FF0DC08295807FAB2BD3
:100C800009F08062672B09F08064452B09F08068C9
:100C900009950895AB2B09F08260672B09F08460F9
:100CA000452BB1F38860F4CF80E0F2CFFC01A08146
:100CB000B1818D91B183A0830895DC01ED91FC9108
:100CC000119784913196ED93FC9308958093D50408
:100CD00008958093D604089521E030E001C0220FEA
:100CE0008A95EAF78091D604822BF3CF21E030E099
:100CF000A90102C0440F551F8A95E2F7CA018095E9
:100D00009091D6048923E5CF292F9A3090F587302A
:100D100080F590E037E0239F800D911D1124282F4E
:100D2000277041E001C0440F2A95EAF723E0969529
:100D300087952A95E1F7FC01EE0FFF1FE80FF91FD9
:100D4000EF54FB4F20E030E070E05191DF01CB0128
:100D5000022E02C0969587950A94E2F781708195DC
:100D60008527842385278E932F5F3F4F23303105BE
:100D700061F70895292F9A3078F5873068F590E06B
:100D800037E0239F800D911D1124682F677023E0A9
:100D9000969587952A95E1F7FC01EE0FFF1FE80F66
:100DA000F91FEF54FB4F40E050E080E0219130E02C
:100DB000062E02C0369527950A94E2F72170332754
:100DC000042E01C0220F0A94EAF7822B4F5F5F4F77
:100DD0004330510559F7089580E008959091D60465
:100DE00021E030E0F90101C0EE0F8A95EAF7D90160
:100DF00002C0AA0FBB1F6A95E2F7EA2B01C0220FBF
:100E00004A95EAF7892F8E23E81303C0892F822B96
:100E100060CF2095822F8923FBCF8091DE049091B3
:100E2000DD04981301C008958F5F8770FACF909109
:100E3000D804809589238093D804282F2770211106
:100E400010C0891771F090911F0592FF0AC0869516
:100E5000869586954BDF1092D8041092DA04109292
:100E6000D9040895982F90958091D3048923809375
:100E7000D30408958091D204811531F01092D204E8
:100E80001092DC041092DB040895803E9105D9F1A4
:100E9000C8F48133910509F482C048F48932910580
:100EA00009F472C08A32910509F480C0089589332B
:100EB0009105E9F082389105D1F08533910509F467
:100EC0005EC00895843E9105D9F148F4823E9105B3
:100ED00039F1833E910549F181EE90E00895863E17
:100EE0009105C9F1873E910509F43EC0089520910E
:100EF0001E052370211164C020911F0523FF14C01B
:100F000089E290E0089520911E0520FD45C03091B2
:100F10001F0530FF09C024FD24C083EE90E0089532
:100F200020911E0522FDF7CF089520911E0522FD78
:100F300044C030911F0530FD43C024FFF5CF11C0E0
:100F400020911F0521FFF0CF80911E0584FD09C06F
:100F500087EE90E0089520911E0523FFE5CF24FF42
:100F6000F7CF80E090E0089520911E0523FD2BC06F
:100F700030911F0531FFE1CF84EE90E0089520917C
:100F80001E0525FFD1CFBCCF20911E0525FD1EC01B
:100F900020911F0523FFC8CF89E390E00895209199
:100FA0001E0526FFC1CF8AE290E0089520911E051C
:100FB00026FFBACF81E390E0089582EE90E0089595
:100FC00080EE90E0089586EE90E0089585E390E04D
:100FD000089590911E0592FF10C041E0282F2471C2
:100FE000243009F040E031E0282F2871283009F042
:100FF00030E0431711F02CE0822793FF10C041E04E
:10100000282F2471243109F040E031E0282F287185
:10101000283109F030E0431711F02CE0822730919D
:101020001F0530FF10C051E0282F2171213009F039
:1010300050E041E0282F2871283009F040E0541793
:1010400011F029E0822731FF10C041E0282F2171E3
:10105000213109F040E031E0282F2871283109F0D2
:1010600030E0431711F029E0822794FD877E089530
:101070001F93CF93DF9309DFEC01811522E59207DF
:1010800008F052C0811540E5940708F0CDC0803EBD
:10109000910520F58D3C910508F0A1C0883A910595
:1010A00070F4853A910508F097C081309105B9F147
:1010B0000497813A910598F1C0E0D0E030C0885A99
:1010C00091094B97C8F7C85AD0E0CC0FDD1FCA581A
:1010D000DE4F0990D881C02DD46421C0811550E421
:1010E0009507B0F4C11580E2D80708F0B3C0C83E38
:1010F000D105A8F0CE019A9581159F41E8F68D2F74
:1011000068DF182FCE019927C0DEEC01D12B07C074
:101110009927BBDECC27DF70C82BD92BD06ACE0134
:10112000DF91CF911F910895803842E59407C8F56B
:10113000803652E5950708F05BC0C03482E5D807D9
:10114000D0F4C03292E5D90708F04BC08C2F8695B9
:10115000869520E2829FC0011124C37021E030E017
:10116000A90102C0440F551FCA95E2F7EA01C82B36
:10117000D92BDD68D4CF8C2F86958695877050E269
:10118000859FC0011124C37021E030E0A90102C095
:10119000440F551FCA95E2F7EA01C82BD92BDC682A
:1011A000BECF803C52E5950758F48F71C03AD245C6
:1011B000A0F590E0982F8827EC01C46FD06AAFCFDC
:1011C000805C9245809708F077CFDC2FCC27CC2726
:1011D000DF71C06FD06AA3CFA497D064A0CFD065D1
:1011E0009ECFCF71D0E0DC2FCC27C16FD06A97CFD4
:1011F00086958695877020E2829FC0011124C37076
:1012000021E030E0A90102C0440F551FCA95E2F762
:10121000EA01C82BD92BDA6882CFDBDEC82FD0E0F9
:10122000DC2FCC27D0627BCF8F71D3DE93E0CC0F45
:10123000DD1F9A95E1F7CC27DF70282F30E084FF7F
:1012400005C050E1859F900111243327C22BD32B79
:10125000D06965CF8D2F8F71BCDE182FCE019927F5
:1012600014DEEC01D12BDECF80E00895F894E82F56
:10127000E295EF70F0E041A18F7021E030E0B9011C
:1012800002C0660F771F8A95E2F7CB01962F9095E3
:10129000942391A392A1892B82A37894089580919D
:1012A0009B04811103C080911A020895E091A70464
:1012B000F091A804309739F00190F081E02D30973B
:1012C00011F00995089580E00895A3E0B0E0EBE601
:1012D000F9E00C94F32A9C01809118029091190274
:1012E00082179307B1F03093190220931802E0910E
:1012F000A704F091A804309761F00084F185E02DF7
:10130000309739F083E089833B832A83CE010196AD
:1013100009952396E2E00C940F2BA3E0B0E0E3E9FB
:10132000F9E00C94F32A9C01809116029091170227
:1013300082179307B1F03093170220931602E091C1
:10134000A704F091A804309761F00084F185E02DA6
:10135000309739F084E089833B832A83CE0101965C
:1013600009952396E2E00C940F2B809101010895DA
:101370002FB7F894609112027091130280911402B9
:10138000909115022FBF08950F931F9380919B0496
:10139000811521F0EDDF1F910F910895E9DF009194
:1013A0009D0410919E0420919F043091A004600F31
:1013B000711F821F931FEFCF87E797E79093010874
:1013C0008093000888E19AE00FB6F894A89580937E
:1013D00060000FBE90936000FFCF08950895FC0158
:1013E0009B0180910802909109028617970740F0AF
:1013F000672B29F48091E8008E778093E800C9017B
:1014000040E0009741F4411106C08091E80082FF5E
:101410002FC080E00895209174042115A9F1253092
:10142000A9F12091E80023FD2DC02091E80022FDC4
:10143000ECCF2091E80020FFE4CF3091F300209121
:10144000F200009719F02830310558F041E02830BB
:10145000310509F040E02091E8002E772093E80064
:10146000D0CF41914093F10001972F5F3F4FE9CFDB
:1014700080917404811541F0853041F08091E8003D
:1014800083FFC3CF81E0089582E0089583E008954B
:101490008091020287FF13C08091E80082FF06C09E
:1014A0008091E8008B778093E80008958091740420
:1014B0008111F2CF0895809174048115D9F3809140
:1014C000E80080FFF8CF8091E8008E77ECCF209184
:1014D000E4003091E50095E6A9012091EC00822F0F
:1014E000817020FF06C08091E80080FF06C080E088
:1014F00008952091E80022FD1AC08091740481159E
:1015000089F0853089F08091EB0085FD0FC0209136
:10151000E4003091E50042175307F9F29A95E1F69D
:1015200084E0089582E0089583E0089581E00895BD
:10153000E8EDF0E080818E7F80831092E2001092CF
:10154000DA001092E100A0EEB0E08C9181608C9303
:1015500080818F77808319BCA7EDB0E08C918E7F5E
:101560008C9380818F7E8083109201020895E09198
:10157000A704F091A804309739F00284F385E02D98
:10158000309711F060E209950895FC01AC014B5FC2
:101590005F4F8FEF61E39191892728E030E0982F2A
:1015A000990F87FF09C0892F862721503040B9F74E
:1015B000E417F50781F70895892FF7CF8091D604B6
:1015C000811531F083FF04C084FF02C085E084CB25
:1015D00085E08CCB982F9093E900891771F070917A
:1015E000EC002091ED005091F00021FD09C09F5FBB
:1015F000973089F78093E9000895762F242F50E0E3
:101600003091EB003E7F3093EB003091ED003D7F59
:101610003093ED003091EB0031603093EB0070932C
:10162000EC002093ED005093F0002091EE0027FD98
:10163000DECF0895A0E0B0E0E0E2FBE00C94ED2AFC
:10164000C8EDD0E088818F7E8883E7EDF0E080816F
:101650008160808384E082BF81E080930102888181
:101660008E7F888302EE10E0F80110821092DA007B
:1016700081EEC82ED12CF601108288818F77888365
:1016800088818068888388818F7D888319BC1092C7
:10169000740410920002109228021092FF0190EE42
:1016A000E92EF12CF70180818B7F80838881816016
:1016B000888342E060E080E08DDFF60180818E7FEC
:1016C0008083F8018081816080838081886080834D
:1016D000F70180818E7F8083888180618883CDB788
:1016E000DEB7E8E00C94092BE091DE049091DD0474
:1016F00027E0E91302C080E00895AE2FB0E02E9FEE
:10170000F0011124E152FB4F3181361306C03081C4
:10171000381303C03581341304C0FD013196E770DE
:10172000E8CF81E00895CF93C82F682F83E090E041
:101730000E94752B8C2FCADACF9108951F93CF93F7
:10174000DF93962F122F632F8430D8F49A30C8F489
:101750004730B8F4C42FD0E0CC0FDD1F2EE0929FAD
:10176000C00DD11D11249CE8899FC00DD11D1124ED
:10177000CE0189960E94752B612FCE018A960E9418
:10178000752BDF91CF911F9108958F929F92AF9209
:10179000BF92CF92DF92FF920F931F93CF93DF936D
:1017A000809072049090730481E090E090937304B1
:1017B00080937204A12CB12C00E0650110E012C0EE
:1017C000FE01259135914F2D612F802FB7DF229695
:1017D000F39487E0F812F4CF87E0C80ED11C1F5FA6
:1017E0001A3039F0E601CC0FDD1FCB50D84FF12C69
:1017F000E7CF0F5F86E4A80EB11C0430F1F690929B
:10180000730480927204DF91CF911F910F91FF902A
:10181000DF90CF90BF90AF909F908F9008950F93DF
:101820001F93CF93DF938B01EA019091740494305E
:1018300051F58093E9008FEF9091E80095FD06C087
:1018400095ED9A95F1F700008A95B1F78091E8003F
:1018500085FF19C03CDE811111C08091E80085FD33
:1018600006C08091E8008E778093E800F3CFF801FE
:1018700081918F018093F100219779F78091E800A1
:101880008E778093E800DF91CF911F910F9108959B
:10189000792F603229F440E250E0682F82E0BFCF18
:1018A0000895CF93DF93D82FC92F48E050E0682FD9
:1018B000792F81E0B4DF88E0ED2FFC2FAAE0B2E0C1
:1018C00001900D928A95E1F7DF91CF910895BC01C7
:1018D00043E050E084E0A3CFA0E0B0E0E2E7FCE02A
:1018E0000C94EB2AF82EE92EB62EA72E8A018091B1
:1018F000F6019AE0C92ED12C8A3018F0CC24C3947A
:10190000D12CC1E0D0E06B2D7A2D8F2D9E2DF801CA
:101910000995811116C02196CC16DD0694F0CC9F56
:10192000C001CD9F900D900D112420E030E045E3E3
:101930004A95F1F700002F5F3F4F28173907B9F795
:10194000E2CFCDB7DEB7EAE00C94072B90911F05EC
:1019500092FB222720F9281771F080FB92F99093CF
:101960001F0560911E0570911F0584E090E00E94A4
:101970008F2B82E05CCA0895CF92DF92EF92FF92A4
:101980001F93CF93DF9300D000D0CDB7DEB7C090C8
:101990008104D0908204E0908304F0908404E8DC19
:1019A0006C197D098E099F0911E064367105810566
:1019B000910568F1E9DCDC01CB010296A11DB11DA6
:1019C00089839A83AB83BC838091290190912A01FA
:1019D0008B579B4F20912801422F50E0253010F06B
:1019E00044E050E0BE016F5F7F4F0E94492B82E0D0
:1019F00090E00E94612A182F811549F0B9DC6093AC
:101A00008104709382048093830490938404812FD3
:101A10000F900F900F900F90DF91CF911F91FF903B
:101A2000EF90DF90CF9008958F929F92AF92BF92E8
:101A3000FF920F931F93CF93DF9300D000D000D07D
:101A4000CDB7DEB7F62E072F80E090E00E94612A26
:101A5000182F811509F45CC080911B01482F50E0BC
:101A6000811511F041E050E060911C0170911D0161
:101A70006B577B4FCE0106960E94492B80909704AE
:101A800090909804A0909904B0909A0471DC681921
:101A900079098A099B09643671058105910530F43D
:101AA00086E894E072DD9E81891791F181E090E0F3
:101AB0000E94612A8115B9F180912301482F50E0DD
:101AC000863010F045E050E06091240170912501CE
:101AD0006B577B4FCE0101960E94492B86E894E01C
:101AE00054DD9E8189131FC043DC6093970470937B
:101AF00098048093990490939A0485E0FE013196AE
:101B0000A2E9B4E001900D928A95E1F781E00CC062
:101B100085E0E6E8F4E0DE01119601900D928A95E9
:101B2000E1F71111EACF80E095E0E2E9F4E0AF2DB2
:101B3000B02F01900D929A95E1F70F900F900F90B2
:101B40000F900F900F90DF91CF911F910F91FF9009
:101B5000BF90AF909F908F9008958F929F92AF9279
:101B6000BF92DF92EF92FF920F931F93CF93DF9379
:101B7000C82F8B01F42ED22ED32FFB0180809180B1
:101B8000A280B380F5DB681979098A099B0964365C
:101B900071058105910510F4F11421F1EC2E0C2E44
:101BA000000CFF0888E0C802F0011124E85EFE4F37
:101BB000818192818B579B4F2081422F50E02115CC
:101BC00011F041E050E06D2D7D2F0E94492BC7019F
:101BD0000E94612A811539F0CBDBF80160837183A3
:101BE0008283938381E0DF91CF911F910F91FF90CA
:101BF000EF90DF90BF90AF909F908F90089541E05D
:101C000090918F048091D604981301C040E026ED96
:101C100034E06DE774E083E0A0DF811571F041E00E
:101C2000909190048091D504981301C040E025ED77
:101C300034E069E774E084E090CF0895A1E0B0E07B
:101C4000E4E2FEE00C94F32A2ADB898341E09091E0
:101C50009104981301C040E09E012F5F3F4F65E75C
:101C600074E085E07ADF2196E2E00C940F2B0F936D
:101C70001F93CF93DF93843030F56A3020F54730DF
:101C800010F5C42FD0E0CC0FDD1F2EE0629FC00DF9
:101C9000D11D11243CE8839FC00DD11D1124CE011C
:101CA00089960E94592B082F10E0102F0027CE0193
:101CB0008A960E94592B9801282BC901DF91CF9158
:101CC0001F910F91089580E090E0F8CF462F672F85
:101CD0002091A3043091A404232B81F4703F39F4A4
:101CE000403F61F48091A1049091A20408957A305C
:101CF00028F4473018F4843008F4B9CF80E090E03D
:101D00000895A0E0B0E0E7E8FEE00C94EE2A7C0144
:101D10000091D6048091D504082BC3E0D0E010E0F8
:101D2000C8010C2E02C0959587950A94E2F780FDB4
:101D300009C02197A8F7D12C8D2DCDB7DEB7E7E0EC
:101D40000C940A2BDC2EB7018C2FC0DF91D90197A0
:101D500081F3F2CF0F931F93CF93FC018581008114
:101D60001181811581F0611571F0C801CADFC82F9A
:101D7000682FC8010E948406B8018C2FA7DFCF917D
:101D80001F910F910895C8010E94BA06C82FF4CF81
:101D9000CF93DF93D82FC92FB4DF6D2F7C2F96DF21
:101DA00067D9DF91CF910895FC018481811599F065
:101DB00080819181EDDF282F92959F70963099F068
:101DC00060F4925F9F70923030F4203FB1F038F4AD
:101DD00081E0283E38F080E008959A5FF3CF81E0FB
:101DE000243FC9F7089591E0213F09F090E081E098
:101DF000283E08F080E0892B089581E00895382F6F
:101E0000292FCB01A32FB22F873A21E09207A105FA
:101E1000B10520F4875A9D4F0C94592B80E008950A
:101E200085E290E00E94592B873289F486E290E0A7
:101E30000E94592B833059F487E290E00E94592B7D
:101E400091E0853209F090E0892F8170089580E05B
:101E5000FCCFCF93DF93682F81E06A3019F06D30AB
:101E600029F480E075D0DF91CF91089580913402FC
:101E70009091350226E0FC01A9EFB1E001900D92AE
:101E80002A95E1F7603E08F458C026E0FC01119263
:101E90002A95E9F7C0913402D091350246E050E02E
:101EA000BE0189EF91E00E943C2B9E0127553240F4
:101EB000892B41F1C90145E0969587954A95E1F74F
:101EC00041E050E0BA0102C0660F771F8A95E2F741
:101ED000CB016091590470915A04862B972BB9015C
:101EE0006B5F7F4FE5E076956795EA95E1F702C075
:101EF000440F551F6A95E2F7842B952B90935A0453
:101F0000809359042A5F3F4F40913602642F70E05E
:101F1000C9010E94CF2A481B463010F4240F311DFE
:101F2000211572E0370710F020E030E0295A3D4FCC
:101F3000309335022093340296CFF6E06F9FB001C4
:101F40001124685B7E4F46E050E00E94332BA2CF05
:101F5000CF93382FE0913402F0913502E755F240EB
:101F600020913602622F70E0CF010E94CF2A281BF9
:101F7000822F311559F066E00E941A2BC82FC150EC
:101F800010F4CF91089580E264DFF9CF8E0F9F2F78
:101F9000911D811522E0920710F080E090E0895AAF
:101FA0009D4F9093350280933402EBCFCF93DF9314
:101FB000EC01FE018491811103C0DF91CF9108955E
:101FC00048DF2196F6CFAB0124E630E0BC0188E77C
:101FD0000E9490289C0181E0232B09F080E0089565
:101FE00080916204811561F080915F04811541F058
:101FF00062E070E086E491E0E6DF811110925F0418
:102000000895809162048115E9F0B2D9DC01CB0119
:10201000805A9541AF4FBF4F80935B0490935C040F
:10202000A0935D04B0935E0480915F0481110AC0A7
:1020300062E070E084E491E0C6DF811519F081E090
:1020400080935F040895A0E1B0E0E9E2F0E10C9430
:10205000E52AFE01319680E1DF011D928A95E9F7BC
:102060000BE110E099E5A92E92E0B92E27EA422E65
:1020700055245394612C712C4F0173016201B1E11D
:102080004B165104610471041CF080E1C82ED12C60
:10209000A601B501C4010E94662BAC0CBD1C0D2C21
:1020A000000CEE08FF084C185D086E087F08015010
:1020B000104019F76096E0E10C94012B6FEF85E278
:1020C00090E00E94752B6FEF86E290E00E94752BE6
:1020D0006FEF87E290E00E94752B60E088E290E06D
:1020E0000E94752B52DBAFDF67E285E290E00E9431
:1020F000752B63E086E290E00E94752B65E287E233
:1021000090E00C94752B1F921FB61F9211248F9391
:102110009F93AF93BF9380912702811113C0809149
:10212000120290911302A0911402B09115024196EF
:10213000A11DB11D8093120290931302A09314026B
:10214000B0931502BF91AF919F918F911F901FBEC9
:102150001F9018952FB7F894809112029091130256
:10216000A0911402B09115022FBF0895CF93DF9371
:10217000C091D3048091D704C82B8091D2048115DB
:10218000F1F0E8DF2091DB043091DC04821B930B3B
:102190008838934110F00E943A07D091D20420E091
:1021A00086EE91E0FC013081019631112F5F31E024
:1021B0008C3E9307B9F721110E943A07CD2BC093AB
:1021C000E40148E050E069EA74E084EE91E00E94A6
:1021D0003C2B892BB9F088E0E4EEF1E0A9EAB4E009
:1021E00001900D928A95E1F7E091A704F091A8047F
:1021F000309741F00280F381E02D309719F084EEA2
:1022000091E00995DF91CF9108951092D304E6EE05
:10221000F1E086E0DF011D928A95E9F780E090E029
:1022200054D880E090E079D81092D7049FCFEDDFAA
:102230002FEF84E39CE0215080409040E1F700C004
:10224000000088E19AE00FB6F894A89580936000AA
:102250000FBE90936000FFCFAAE2B0E0E2E3F1E1AD
:102260000C94F22A82E092E0FC0101962091F100A8
:10227000208322E08A309207B9F7809103028930E7
:1022800009F457C0C8F4823009F4B2C0833009F4AD
:1022900082C0813081F18091E80083FFE6C08091A7
:1022A0000202909103029A3008F0DFC0E92FF0E0BB
:1022B000EB55F44D0C94262B8A3009F489C08B30F1
:1022C00051F780910202813231F78091060290919C
:1022D0000702892B01F78091E800877F8093E8004F
:1022E000D7D881E090910402911101C080E08093E1
:1022F00002018BDFD0CF80910202813A61F680919A
:10230000E800877F8093E8008091060290910702A1
:10231000892B59F060E080E090E070E060D8809117
:10232000E8008B778093E800B6CF68E08AE092E01F
:10233000F4CF80910202813209F0ADCF8091060284
:10234000909107028D7F892B09F0A5CF8091E8003D
:10235000877F8093E8008091E80082FF17C090910A
:10236000F3008091F200029731F48091F100813006
:1023700011F0863021F48091F10080930101809169
:10238000E8008B778093E80083D885CF8091740430
:102390008111E1CF80CF80910202813A09F07BCF99
:1023A0008091060290910702892B09F074CF8091E9
:1023B000E800877F8093E8008091E80080FFFCCFF1
:1023C000809102018093F1008091E8008E77DACF4E
:1023D00080910202813209F05ECF8091E800877F10
:1023E0008093E80055D8809105028093000153CF77
:1023F00080910202813A09F04ECF8091E800877FF8
:102400008093E8008091E80080FFFCCF809100017C
:10241000D9CF803889F0823841F5809106028F70DB
:10242000873018F58093E9008091EB0085FB8827C1
:1024300080F91092E90006C080912802880F9091DF
:10244000FF01892B9091E800977F9093E80080939B
:10245000F1001092F1008091E8008E7723C0811185
:1024600016C080910402813011F18091E80083FF51
:102470000AC08091E800877F8093E8008091EB009C
:1024800080628093EB00AA96E3E00C940E2B8230DE
:1024900061F780910402811589F01092E900809122
:1024A000E800877F8093E8000E94480ADECF81E041
:1024B000933009F080E080932802EFCF80910602EC
:1024C0008F702FEF280F263080F68093E90020913F
:1024D000EB0020FFE2CF933031F48091EB0080627B
:1024E0008093EB00DACF9091EB0090619093EB003A
:1024F00021E030E0A90102C0440F551F8A95E2F7A0
:102500004093EA001092EA008091EB008860E8CFE7
:102510008111ABCF109104021F778091E300807886
:10252000812B8093E3008091E800877F8093E8000F
:102530000E94480A8091E80080FFFCCF8091E30070
:1025400080688093E30083E0111101C082E08093F2
:1025500074048BCF8058823008F087CF80910402BA
:10256000909105028C3D53E0950799F583E08A83AD
:102570008AE289834FB7F894DE01139620E03EE0AB
:1025800051E2E32FF0E050935700849120FF03C005
:1025900082958F703F5F8F708A30C8F0895C90E0C1
:1025A0008D939D932F5F243161F74FBF8091E80099
:1025B000877F8093E8006AE270E0CE0101960E9476
:1025C000EF098091E8008B778093E8004ECF805D23
:1025D000E6CF292F33272330310509F44EC078F593
:1025E0002130310509F488C08BE590E0E8E3F7E09D
:1025F0002230310509F039CF2091E800277F209360
:10260000E80020910802309109028217930708F42C
:102610009C0140E02115310509F073C0411171C0E2
:102620008091E80082FDCDCF80917404811549F23C
:10263000853039F28091E80083FFF2CFC2CF8091DC
:102640000602909107022132310509F446C0223278
:10265000310509F00ACF8330910508F006CFFC015F
:10266000EE0FFF1FEC5AFE4F0190F081E02D8F5AC4
:102670009E4FDC018C9190E010C09C01332782308A
:1026800021F12330310568F4232BB9F4E1EFF7E0B1
:10269000E4918E2F90E0E1EFF7E0009709F4E5CEAA
:1026A000ABCF2330310509F0E0CEE5EAF7E0E49165
:1026B0008E2F90E0E5EAF7E0F0CFEBEDF7E0E49164
:1026C0008E2F90E0EBEDF7E0E8CFE3ECF7E0E4915C
:1026D0008E2F90E0E3ECF7E0E0CF8330910508F037
:1026E000C4CEFC01EE0FFF1FE65AFE4F0190F081B1
:1026F000E02D89E090E080CF82E190E0E3E9F7E02F
:102700007BCF80917404811509F45BCF853009F487
:1027100058CF8091E80083FD54CF8091E80082FD7E
:102720007FCF8091E80080FF75CF9091F30080917A
:10273000F2002115310519F08830910550F041E083
:10274000089709F040E08091E8008E778093E800D8
:1027500061CF44914093F1003196215031090196A7
:10276000E8CF803809F081CE8091E800877F8093A0
:10277000E800809100028093F1006DCE811175CE4A
:1027800010910402123008F070CE8091E800877F2B
:102790008093E800109300020E94480A1115F9F096
:1027A00084E08093740442E061EC81E00E94EA0AD4
:1027B00042E261EC84E00E94EA0A42E261EC82E0DB
:1027C0000E94EA0A42E260EC83E00E94EA0A8091F9
:1027D0007404843051F482E08093030146CE8091EA
:1027E000E30087FDDDCF81E0DCCF81E0F5CF0F9303
:1027F0001F93CF93C82F811531F18CEF8C0F813A45
:1028000098F506EE11E0F8018191C81701F121E079
:10281000EC3EF207C9F7EFEF80E0D8019D918D0102
:10282000C91781F0EF3F19F4911101C0E82F8F5FB4
:10283000863099F7EF3F31F00E2E000CFF0BEC5174
:10284000FE4FC28393DCCF911F910F910895E6EE66
:10285000F1E08191C81302C0DF011E9231E0EC3E2D
:10286000F307B9F783DCD7CF80E28C0F883068F4A8
:10287000C77081E090E001C0880FCA95EAF7C09167
:10288000D304C82BC093D304DDCF8BE58C0F8330EA
:1028900038F42C2F2452330BC9010E946509D3CF81
:1028A000C85ACB3180F6EC2FF0E0EE0FFF1FE45555
:1028B000FE4F808191810E948D09C5CF811569F1FC
:1028C0009CEF980F913A60F4E6EEF1E09191891354
:1028D00002C0DF011E9291E0EC3EF907B9F746CC49
:1028E00090E2980F983050F4877091E001C0990FF2
:1028F0008A95EAF7892F0E943207F1CF9BE5980F5E
:10290000933020F480E090E00C946509885A8B3174
:1029100020F480E090E00C948D0908951F93CF93EC
:10292000DF93182FEB0163DF209731F4812FC6DF8F
:10293000DF91CF911F9108958FE99FE00197F1F703
:1029400000C000002197F0CFA0E0B0E0EAEAF4E197
:102950000C94EA2A8C01B62EA72E8B2D9A2DF80105
:1029600009958115D1F1813009F051C08B2D9A2D37
:10297000F8010995813061F48B2D9A2DF8010995A4
:1029800060E570E0893311F060E070E0C7DFE5CF0B
:10299000823031F48B2D9A2DF801099528DFDDCF97
:1029A000833031F48B2D9A2DF801099587DFD5CF2F
:1029B000843089F48B2D9A2DF8010995C0E0D0E080
:1029C0009AE0F92E482F4053550B9A014A30510591
:1029D00048F02097A1F48111C0CFCDB7DEB7EBE06E
:1029E0000C94062BFC9EC001FD9E900D1124E90164
:1029F000C80FD91F8B2D9A2DF8010995E3CFEFE968
:102A0000FFE03197F1F700C000002197E2CFE82FF7
:102A1000F0E0E854F94F9490282F269526952695B6
:102A200030E0F901E855F94FE4908770F12C082E59
:102A300002C0F594E7940A94E2F7E0FAEE24FF244A
:102A4000E0F8F901E856F94FC490D12C082E02C0E5
:102A5000D594C7940A94E2F7C0FACC24DD24C0F8D8
:102A6000F901E857F94FC491D0E002C0D595C79558
:102A70008A95E2F7C170DD27E114F10411F081EECF
:102A8000B6DEC114D10411F086EEB1DE60E070E074
:102A9000892D44DFC114D10411F086EE0FDFE1145B
:102AA000F10411F081EE0ADFCD2B09F456CF60E07E
:102AB00070E08CE26BCF811531F09091D304892BBB
:102AC0008093D30453CB0895811519F00E943207E7
:102AD0004DCB0895811531F09091D704892B8093C7
:102AE000D70444CB0895811539F080959091D7048F
:102AF00089238093D7043ACB08958091CD04811522
:102B000021F082E2F0DF1092CD040895962F2091FB
:102B10001F0522FF0FC0682F660F660F660F692B17
:102B20006093D8040E946C0615DB9093DA048093BE
:102B3000D90408950C946C069091D204292F28236F
:102B4000211559F0809589238093D204811531F0A5
:102B500001DB8093DB049093DC04089580E090E037
:102B6000F8CFCF93DF93EC01F5DA8C1B9D0BDF914F
:102B7000CF910895EF92FF920F931F93CF93DF931E
:102B8000C62FD42F122F811599F06093D104E2DA69
:102B90009093F8018093F701C77081E001C0880F1E
:102BA000CA95EAF788DFCDB7DEB7E6E00C940B2BC9
:102BB0008091D10468132FC0E090F701F090F801E4
:102BC000C9DA8E199F098436910528F500E20D0FA8
:102BD000CD1799F0C770FF24F3948F2D01C0880F93
:102BE000CA95EAF771DF083040F48D2F877001C075
:102BF000FF0C8A95EAF78F2D5EDF60E070E0812F91
:102C00008DDE083080F6D77081E001C0880FDA953C
:102C1000EAF75ADFC8CFC77081E001C0880FCA95B4
:102C2000EAF7F7CFA7E0B0E0E8E1F6E10C94E32A99
:102C30008C01FC018481811509F44AC061E0C8015E
:102C400089D87C018132F8E79F0791F1FC01E054BB
:102C5000FE47E930F10520F4E155F44D0C94262BA4
:102C6000F80145814111A4C023E7E2162CE7F206E2
:102C7000F9F0E2EAEE16E2E5FE0609F4B8C108F062
:102C80008EC1C70190528115904208F4A3C1F1EEA4
:102C9000EF16F10409F4ABC125EEE216F10483C18D
:102CA000F8018581811521F081E090E00E94930B6D
:102CB0008091D8048770811559F0F80185818115BC
:102CC00039F080911F0582FF03C082E00E94170740
:102CD0002796E2E10C94FF2AF8018581811541F3E2
:102CE00082E090E0E3CFF8018581811509F384E06B
:102CF00090E0DCCFF8018581811559F08091CC04FA
:102D0000811103C081E08093CC0483E00E946C06B3
:102D100005C01092CC0483E00E9476060E94DE0A71
:102D2000C7CFF8018581811549F08091CC048111CC
:102D300003C081E08093CC0484E0E8CF84E00E946B
:102D400076061092CC04EACFF8018581811521F036
:102D500085E00E946C06ACCF85E00E947606A8CF85
:102D6000F8018581811591F080911E0582FD03C0D7
:102D700081E93DDD9DCF8FE09CE09A838983BE0190
:102D80006F5F7F4F8DE596E0DFDD92CF81E996DDC5
:102D90008FCFF8018581811549F080911E0582FD54
:102DA00002C080E9E6CF87E09CE0E7CF80E9EFCF83
:102DB000C70197578038910508F008C5BE2CF0E18F
:102DC000EF1608F075CF66EA71E080E090E017D862
:102DD00081116ECFC12CD12C7601B11045C0AE014E
:102DE0004F5F5F4F1A01F10124E011922A95E9F734
:102DF000460157013FEF831A930AA30AB30AC7019A
:102E0000B6010E94FF0E8983811509F451CF8130EC
:102E100009F0ADC02601370142E0440E511C611C8F
:102E2000711CC501B4010E94FF0E8F838A83811536
:102E300009F43ECF8150833060F5C301B2010E9496
:102E4000FF0E8B83811541F03E822D82BE016B5FA8
:102E50007F4F86E596E078DD4601570153E0850E09
:102E6000911CA11CB11C4AC027EAC21621E0D2065F
:102E7000E104F10409F41CCFC701B6010E94FF0E62
:102E80003FEFC31AD30AE30AF30A8111EDCFBA94D4
:102E9000A4CF8F8185508330A0F54601570183E090
:102EA000880E911CA11CB11CC301B2010E94FF0E2F
:102EB0008B83811519F1C501B4010E94FF0E8C832B
:102EC0008115A9F0AB80BC8091E0A9169FEFB906EF
:102ED00010F0BA2CAA24EF81E63039F0E73011F077
:102EE000C501BCD6C501ECD602C0C501B7D64601A6
:102EF000570154E0850E911CA11CB11C75016401A1
:102F000072CFFF8153014201F430C1F7C301B20116
:102F10000E94FF0E782E4601570124E0820E911C7C
:102F2000A11CB11CC701B6016D5F7F4F8F4F9F4F32
:102F30000E94FF0E711409F4BBCE811509F4B8CEBE
:102F40008150990B4FEF489F9001499F300D1124FC
:102F5000472D4150550B240F351F2150310970F278
:102F60008FE99FE00197F1F700C00000F6CF3E82A5
:102F70002D82BE016B5F7F4F86E596E0E5DCBECF1C
:102F80001092D3040E943A07E5D888579C4E90933C
:102F9000CF048093CE0481E08093CD0489CE32EBC0
:102FA000E31632E5F306D9F525EE30E02770332736
:102FB00081E090E001C0880F2A95EAF72091D004C3
:102FC0003091CD043115D9F04115A1F0282B209373
:102FD000D0046ECEF8018681803108F58F2D9927B7
:102FE0008F7199278230910511F04297DCCF21EE45
:102FF00030E0DCCF809582238093D00459CE322FED
:103000003823311561F0982F909592239093D00436
:103010000E943207F8018581811509F449CE80911B
:10302000CD04811509F4D2C0C090D304D090D2044D
:1030300091D888579C4E9093CF048093CE04F8018A
:103040008581811509F4C2C08D2D8C298D7981115E
:1030500095C0E114F0E5FF0600F5E11420E4F20666
:1030600008F09EC036EEE316F10409F43FC0C70134
:1030700090528115904208F099C0F8018681803104
:1030800008F473C0C70199271092D7048D329105B7
:10309000B9F482E08093D7048DC0F4EBEF16F2E52B
:1030A000FF0621F108F052C030E4E31632E5F306E2
:1030B000B8F4E11442E5F406C8F41092D704C7014D
:1030C0008E32910508F08FC08832910508F070C0EB
:1030D0008E31910508F06EC004974A97D0F24EC029
:1030E000C701805692458034910538F7F8018581F3
:1030F000811509F461C31092D104F7E7EF16FCE7DC
:10310000FF0609F492C028E7E2162CE7F20609F45C
:1031100095C09701205E32452032310508F094C0F9
:103120008111ADC03E2D3F7181E090E0AC0102C045
:10313000440F551F3A95E2F77A01642F83E090E03F
:103140000E94752B8E2D0E946606B2CD50EEE516BC
:1031500052E5F50628F480ECE81682E5F806ACCFD7
:10316000C70187579C470297C0CF8F2D8F7184313D
:1031700009F4BCCF863159F41092D704BEDC80919B
:10318000D3049091D004892B8093D3041FC0B5DC65
:103190008091D3049091D004892B8093D304A6CF3F
:1031A000F8018681803108F06DCFA0CFC7016CCFC8
:1031B0008A9721F78091D004811531F08091D7044E
:1031C00092E089278093D7040E94B610F801858188
:1031D000F701E851FC47E730F10508F087CFE854E4
:1031E000F44D0C94262B8C34910521F38D329240B2
:1031F000E0CF26E241EE61EEBDDC5ACD27E245EE9E
:1032000065EEFACF26E241EE60EEF6CF27E245EE1C
:1032100064EEF2CF26E241EE62EEEECF27E245EE1B
:1032200066EEEACF28E241E0EBCF81E00E946C0637
:1032300043E062E081E00E94EE063ACD811511F094
:1032400082E0F4CF82E0BFC28115C9F05AE5E516ED
:103250005CE7F50609F4A6C008F07BC091E0E9162A
:103260009CE7F90609F49CC0E3E0EE16ECE7FE06E5
:1032700009F490C0E114FCE7FF0609F47EC0F801F0
:103280008581C080D180811509F490C0C6010E945B
:10329000810EF82E682FC6010E948406B6018F2D7C
:1032A0000E94660E0E943808D82EF92EF801B580CB
:1032B000A680A2942FE0A2228091D8048770811565
:1032C00009F1CB2CB114F9F0892F807F803469F09B
:1032D00080E28D0D8830B0F0892F807E803229F415
:1032E000F2E0DF1678F0A11469F080911F0582FFEB
:1032F00009C082E00E9417078091D8048770CC240F
:10330000C3948111C12C8F2D82958F70883009F460
:1033100052C108F06BC0843008F04DC02F2D2F70C3
:10332000E22E823008F473C08F2D807F803219F036
:10333000E29480EFE822D11409F4A0C051E0D51640
:1033400009F4FDC0B11409F408C1A11409F4B2C014
:1033500075C02BE5E2162CE7F20631F180911F05CE
:10336000002482FF0394802D3CE5E3163CE7F3063E
:1033700009F085CF0E94A60C82CF0E9405114FEF65
:1033800054E38CE0415050408040E1F700C0000021
:103390000E94DC096FEF7FEF80E090E00E948F2BAE
:1033A0000E94171181E0E6CF80E0E4CFC6010E94C1
:1033B000BA06F82E73CF843009F4E0C0C11409F4C2
:1033C0002AC18091D80480FD26C1F8011582869516
:1033D000869586950E946C06C80124DC8091D804ED
:1033E0008695869586950E94760615C1893009F4E2
:1033F00057C18A5F8F70823008F732EFD31261C1F4
:103400008F2D8F71B1105AC10E946C0602C140E12C
:10341000F41618F0E29490EFE922B114B9F0E11437
:1034200069F080E28D0D883010F0D11009C08091D4
:10343000D3048E298093D3040E94B6108D2D2EC004
:103440008091D7048E298093D704F6CF8D2D36DA5C
:10345000E11409F4B3CF80E28D0D883010F0D11063
:1034600004C08E2D0E94320706C0E0948091D704DC
:103470008E218093D7040E94B610A0CF80911F05A3
:1034800082FD14C0B11461F0E11439F08091D304CD
:103490008E298093D3040E94B61080E0A8D98ECFE5
:1034A00080E00CDAE11409F489CFDBCFB11459F1D3
:1034B000A11003C08E2DFFDA81CF81E0A81211C0C8
:1034C000F090D2048E2D8F21E81609F477CF0E9458
:1034D000AA109093DC048093DB04FE28F092D204BF
:1034E0006DCF95E0A9126ACF8E2DE5DA8E2D24DB03
:1034F0008091D4049E2D9823E91609F45FCF8E297C
:103500008093D4045BCFA11010C08E2DDDDA8E2DF8
:1035100013DB8091D4049E2D9823911509F44ECF8E
:10352000E094E822E092D40449CFE1E0AE1246CF25
:103530008091D3048E21811509F440CFE6CFB114D8
:1035400029F0F6E0AF1608F039CFB4CF25E0A21687
:1035500008F034CF8E2DB8DA31CFA114D9F339E386
:10356000D31209C04FEF57EE83E0415050408040E6
:10357000E1F700C000008D2DA1D920CF8F2D8695B9
:1035800086958370811569F0813009F017CF8D2DF4
:103590009F2D9370B11002C080E090E00E948D09D1
:1035A0000DCF8D2D9F2D9370B11002C080E090E063
:1035B0000E94650903CF8F2D8370811139C0B1102E
:1035C00028C04D2D429546954770440F440F8D2DD0
:1035D0008F70042E01C0880F0A94EAF72D2D2071F8
:1035E000D4FE07C02FE030E001C0220F4A95EAF771
:1035F00020953F2D3695369533703230A1F033301B
:1036000081F04091D504313059F0822B84230E94FF
:1036100066060E944F0960E0C8010E94AA0E58CBBE
:10362000842B822BF4CF822B9091D5048927EFCF66
:10363000B11459F1F0FEEDCF4D2D429546954770EE
:10364000440F440F8D2D8F70042E01C0880F0A94F3
:10365000EAF72D2D2071D4FE07C02FE030E001C025
:10366000220F4A95EAF720953F2D3695369533700F
:10367000323089F0333069F04091D604313041F076
:10368000822B84230E946906C4CF823010F2D4CFEB
:10369000842B822BF7CF822B9091D6048927F2CFEF
:1036A0009F2D9F70F92EB11431F0892F0E946C0666
:1036B0008D2D01DAAECF8D2D07DA8F2D0E94760683
:1036C000A8CFE3EFDE1678F4F0EFDF16D9F021EFA4
:1036D000D21699F0B11409F45EC0A11409F458C0CF
:1036E0008D2D85D896CF33EFD316F1F044EFD41259
:1036F000F1CF80911F0582FD23C08F2D8F71B114F2
:10370000E9F282CEB11469F055E0A51608F081CF38
:103710002F2D2F7181E090E001C0880F2A95EAF7E4
:10372000BBCF86E0A816F2CF80E0B11409F4AACF8F
:103730009F2D9F7181E001C0880F9A95EAF7A2CF73
:10374000B114B9F08091D8048770843049F4109294
:10375000D8041092DA041092D9048F2D8F71AECF55
:1037600095E063E0A91608F054CF8F2D8F71CED964
:1037700050CFE5E0AE1640F01092D8041092DA0473
:103780001092D90464E0F1CF81E00E94170741CF85
:103790008F2D8F7139CEA11401F3F9E3DF1209C027
:1037A0002FEF37EE43E0215030404040E1F700C0BA
:1037B00000008D2D83D82DCFF7E7EF16FCE7FF062D
:1037C00009F0A1CC81E00E94760632CD33E7E31602
:1037D0003CE7F30609F04DCA8091CD04811509F448
:1037E000CFCB8BD965CA80911D05803178F480914B
:1037F0001C05811559F0E091DE042091DD04309123
:1038000018054091170557E02E1301C008956E2F3B
:1038100070E05E9FF0011124DF01A152BB4F1496AE
:103820008C911497811551F111968C9111978313F6
:1038300025C08C91841322C015968C911597811107
:103840001DC012968D919C91A0911905B0911A05F9
:103850008A1B9B0B8436910588F480911D058F701F
:10386000806180931D05EB51FB4F80818F708061DB
:10387000808387E195E0D6D90C940D07FB01319642
:10388000E770C2CFADE0B0E0E8E4FCE10C94E72AD9
:103890008C0186E0F801DE01189601900D928A9560
:1038A000E1F7F801F580848197E1892E95E0992E62
:1038B00060901B05611017C0811591F0F11409F497
:1038C000F9C0C8010E94D40E811509F4F3C087E045
:1038D000F801A7E1B5E001900D928A95E1F783DF49
:1038E000FF24F39455C07080A280B380D0901C0553
:1038F0002091190530911A05A501421B530BD114D3
:1039000009F4BBC04436510508F076C0811541F377
:1039100080911805C180E0901D0550E1E51608F082
:1039200057C0C81214C080911705871110C0F1103C
:1039300049C08E2D8F70806180931D0587E195E0D1
:1039400071D980911D05F8018683F12C21C0F110F9
:1039500039C040E06C2D872D0E94740B40E06C2D27
:10396000872D0E94740BF82E8111EFCF88859985E1
:103970000E94C80E292F22952F70903470F49F70EA
:10398000223098F09115A9F0F8019681903188F4D1
:103990008F2D2D96EEE00C94032B2A5F2F70223092
:1039A00060F0C8013FD9FD2CF3CF911511F08115BE
:1039B00079F3805E883060F3F4CF803F48F3815F15
:1039C0008330F9CF80911D05816080931D05BDCFA7
:1039D000C81238C080911705871134C0F11032C069
:1039E000E682C8011FD987E0F801A7E1B5E00190A0
:1039F0000D928A95E1F774CFE0901D05F0E1EF1686
:103A000048F487E195E00ED987E0F40111928A9598
:103A1000E9F79BCF811509F463CF90911805F80160
:103A2000818198130FC08091170587110BC0F11089
:103A300009C0E682C801F6D887E0F40111928A95A0
:103A4000E9F74ECFC8010E94D40E811599F1F11407
:103A500089F180911D05803208F439CF80911705D6
:103A6000909118059A838983BC82AB826D821E82F5
:103A7000EF82CE010196D6D82ACF4436510520F6E2
:103A8000811509F42DCFF114A9F0909118058181C9
:103A9000981306C080911705871102C087E0A5CF53
:103AA000C8010E94D40E811112CF80911D05816042
:103AB00080931D05C801B6D813CFABE1B0E0E3E6B3
:103AC000FDE10C94F12A4E8B5F8B688F798F8A8F82
:103AD000192F9B8F91111092D7041D8A86E0FE0149
:103AE0007696DE011F9601900D928A95E1F70A8D78
:103AF00080911F0582FF1FC00E94AA102091D90447
:103B00003091DA04821B930B8838934138F080910E
:103B1000D80482FD03C082E00E9417070E94AA1009
:103B20002091DB043091DC04821B930B8838934195
:103B300010F00E943A07011561F00B8B1C8B61E0BD
:103B4000CE010F960E94AA0E61E0CE010F960E9450
:103B5000AA0E0B8B1C8B87E0FE013F96DE011896A8
:103B600001900D928A95E1F7CE0108968BDE8111C6
:103B700010C02091DD043091DE0487E0FE0138960C
:103B8000DE01119601900D928A95E1F78C858111E5
:103B90000BC017E08091DE049091DD0489132BC0E7
:103BA0006B96E4E00C940D2B822F90E001968770C9
:103BB00099273817190671F40E9405111092DD0437
:103BC0001092DE0487E0E7E1F5E0DF011D928A95BF
:103BD000E9F7DFCF97E0929FD0011124A152BB4FAC
:103BE000FE01319601900D929A95E1F78093DD04E4
:103BF0000E940D07CECF189FC001112481529B4F08
:103C000041DE811569F28091DE0490E001968770B3
:103C100099278093DE04BECFA6E0B0E0E2E1FEE1AA
:103C20000C94F12A0E94AA108C018091A504909115
:103C3000A6048017910771F019821A820E94AA10B7
:103C4000BC0149815A8180E090E037DF1093A604DF
:103C50000093A5042696E4E00C940D2BA6E0B0E0BA
:103C6000E4E3FEE10C94F12A8C019093A20480938A
:103C7000A104011580E21807B0F4C801805E910923
:103C8000089728F06AE675E10115110511F46BE556
:103C900075E1C8010E942A06802F0E94F71326961C
:103CA000E4E00C940D2B80EF89838A830E94AA1094
:103CB0008160BC0149815A8181E091E0FEDEEFCF55
:103CC000A6E0B0E0E6E6FEE10C94F12A8C019093C8
:103CD000A2048093A104011580E21807B0F4802F9C
:103CE0000E945E14C801805E9109089728F063E77E
:103CF00075E10115110511F464E675E1C8010E9432
:103D00002A062696E4E00C940D2B80EF89838A83A3
:103D10000E94AA108160BC0149815A8181E090E033
:103D2000CCDEEFCFAFE0B0E0E8E9FEE10C94E62AAC
:103D3000FE0131968AE0DF011D928A95E9F780E65F
:103D4000E82E81E0F82E8F0195E6C92E91E0D92E5C
:103D50003F01AA24A394B12C3CE6832E31E0932E9C
:103D6000F70181917F018F3F09F43EC0F894E82F5D
:103D7000E295EF70F0E021A18F70A50102C0440F21
:103D8000551F8A95E2F7CA01922F982B91A392A111
:103D90008095892382A3789400C0E5E6F1E031E0C4
:103DA000512C21912F3F79F0A22FA295AF70A05EE8
:103DB000B0E08C9190E02F7002C0959587952A9580
:103DC000E2F780FF87C080E0582A330F8E169F06E7
:103DD00041F7F70182918F3F11F00E94360950EAB6
:103DE0005A95F1F7D8015C920F5F1F4FCE14DF0494
:103DF00009F0B6CF4AE050E0B3018BE192E00E94B7
:103E00003C2B9C01892B41F08AE0F301ABE1B2E04D
:103E100001900D928A95E1F70091260210E0085971
:103E20001B4F232B09F458C081E08093F5010E94B9
:103E3000AA109093F4018093F30180919B04811563
:103E400009F4A4C07E01BBE0EB0EF11C85E0F70194
:103E500011928A95E9F78091F6018A3008F060C0E6
:103E600044E15DE0B701C8010E946C0C811509F4C2
:103E70007BC04CEB5CE0B701C8010E946C0C811563
:103E800009F472C04FEF5DE0B701C8010E946C0CED
:103E9000811509F469C04EE15EE0B701C8010E94D6
:103EA0006C0C811509F460C01092F6018091250216
:103EB00090E045E050E0B70188599B4F0E943C2BB1
:103EC00021E02093F201892B09F041C02F96EFE009
:103ED0000C94022B832F78CF8091F501811509F482
:103EE000ACCFE090F301F090F4010E94AA108E197B
:103EF0009F09059708F4A1CF45E050E06BE172E01F
:103F0000C8010E943C2B892B41F085E0EBE1F2E0F7
:103F1000D80101900D928A95E1F71092F5018DCFAD
:103F2000C090F001D090F1010E94AA108C199D0957
:103F3000843F914008F094CF8091F201811531F2D5
:103F400085E0D7011D928A95E9F71092F201A091C0
:103F50002502B0E0A859BB4F85E0FE013B960190D9
:103F60000D928A95E1F7B2CF8091F6018F3F39F437
:103F70000E94AA109093F1018093F001DDCF8F5F32
:103F80008093F6018A3008F491CFF2CF85E0F801F2
:103F9000A6E8B4E001900D928A95E1F786E894E0F6
:103FA0000E94C50A80938504C0908B04D0908C0435
:103FB000E0908D04F0908E048091EC019091ED01E1
:103FC000A091EE01B091EF01C816D906EA06FB06F2
:103FD000B1F0C092EC01D092ED01E092EE01F092CE
:103FE000EF010E94B809C61AD70AE80AF90AC09276
:103FF0009D04D0929E04E0929F04F092A0048091D0
:104000008F048093D604809190048093D50480918E
:10401000910480931A025ACFCDB7DEB7AA970FB694
:10402000F894DEBF0FBECDBF85B7806885BF85B76A
:10403000806885BF84B7877F84BF0FB6F894A89542
:1040400080916000886180936000109260000FBED4
:1040500080E890E00FB6F89480936100909361003F
:104060000FBE81E08093030184E399E09093E30124
:104070008093E2010E94980A0E941A0B8091E2004C
:1040800084608093E200789480917404811599F0A3
:104090008091E9001091EC008F701795112717950A
:1040A000182B1092E9008091E80083FD0E942C11EA
:1040B0001F701093E90082E084BD93E095BD9AEFF4
:1040C00097BD80936E0010929D0410929E041092F2
:1040D0009F041092A0040E94100F811102C00E9440
:1040E0005E108091D80080618093D8002AE12A95E3
:1040F000F1F700C08091D900182F117080FD04C025
:104100000E94980A1092740410939B0410939C04CC
:104110001093040111110E947C2980910401809167
:10412000040190E0811101C095E09093260285E0A2
:10413000891B8093250200E611E0A5E6EA2EA1E0A6
:10414000FA2ED8018D918D018F3F11F00E94360912
:10415000E016F106B1F705E611E0F80181918F0153
:104160008F3F11F00E943609F1E00C361F07A9F7C6
:104170008AE0E8E6F4E0DF01282F1D922A95E9F7AE
:10418000EBE1F2E0DF011D928A95E9F780E090E033
:104190000E94612B833E9E4F21F40E94100F8111DB
:1041A00029C063EE7EEF80E090E00E948F2B60E0FC
:1041B00082E090E00E94752B81E08093D50461E05D
:1041C00083E090E00E94752B60E074E184E090E071
:1041D0000E948F2B0E945E1040E050E0BA018FE0F9
:1041E00090E00E94872B40E050E0BA0183E190E02C
:1041F0000E94872B82E090E00E94592B8093290235
:1042000084E090E00E94612B90931F0580931E052F
:1042100089DDEFEFF6E721E0E150F0402040E1F7E3
:1042200000C000007FDD8091680480FF08C06FEF50
:104230007FEF80E090E00E948F2B0E94DC0983E0FA
:1042400090E00E94592B0E9466061092570480E865
:1042500080933602E6D66BE070E08CE39AE00E9431
:10426000E30F811509F43FC08091570465E070E0C9
:1042700081FD98C087E39AE00E94E30F811599F1D0
:104280006DE070E085E29AE00E94E30F811559F13C
:104290000E94B809DC01CB01805A9541AF4FBF4F56
:1042A00080935B0490935C04A0935D04B0935E04E0
:1042B000E7E5F2E080E092E0DF019C011D922150F1
:1042C0003040E1F7F0933502E09334028FEF9FEF37
:1042D00090935A048093590481E080936204809300
:1042E0005F041092580480919B04811102C00E94C7
:1042F0007F2985E091E09093A8048093A7048091A2
:10430000740410E4853009F484C00CDD0AE212E084
:10431000F8E6EF2EF4E0FF2ED701F80191918D9190
:1043200024E332E02E173F0709F47DC09817B1F35C
:1043300080909B04D12CD701CD907D01F801919004
:104340008F019C1431F19C24B12CAA24A394892DB3
:104350008A218115B9F08114A9F0B982DA820E940C
:10436000AA109C838B83F1E0FD8391E08C2D8A2140
:10437000811101C090E09E8349815A816B817C81CB
:104380008D819BDBB394AA0C27E0B212E0CFF80139
:10439000C292D3943AE0D312CECF0E94C409DD2456
:1043A000D39445C082E39AE067CF8091740484304F
:1043B00029F10E94F00F1092270288E190E00FB6D9
:1043C000F894A895809360000FBE1093600083B7A7
:1043D000817F846083BF83B7816083BF7894889531
:1043E00083B78E7F83BF0FB6F894A8958091600045
:1043F000886180936000109260000FBE93DCE8E655
:10440000F4E08191811145C4A2E7B4E0AE17BF0783
:10441000C1F780917404853009F4C7CF0E9405115B
:104420000E944F0972CF981383CFF6DBD12C809175
:104430009B04811589F08091CD04811569F00E945B
:10444000AA102091CE043091CF04821B930B8F3F92
:104450009F4710F40E947D1580916204811509F434
:1044600058C000916004109161040E94AA10801B42
:10447000910BC29770F10E94AA10909361048093EF
:10448000600487E592E090933502809334020E94A5
:104490004F09182F83EA9AE010FD02C08BE99AE0D9
:1044A0000E94D60F86E99AE011FD02C081E99AE0E8
:1044B0000E94D60F8CE89AE012FD02C087E89AE0CD
:1044C0000E94D60F81E00E94A80F87E49AE00E9424
:1044D000D60F8091590490915A04892B09F063C03A
:1044E00080915F048115A9F00E94B80900915B04D6
:1044F00010915C0420915D0430915E04601B710B8F
:10450000820B930B6F3F7F4F8F4F9F4710F40E949A
:10451000F00FD1100E9401100E944F099091630486
:10452000891721F0809363040E94B8098091740474
:10453000843009F0E4CE83E08093E9008091E800C4
:1045400082FFDDCE8091E80090E085FF06C00E94EA
:10455000670A811509F4F8C091E08091E8008B7733
:104560008093E800911509F4CACE0091A30410913C
:10457000A404E9810115110509F403C1EE3F09F016
:1045800023C18A81833020F08550833008F01CC11C
:10459000EA81EE3008F018C1F0E0E154F44DCE01AC
:1045A00001960C94262B80916204811509F498CF12
:1045B00080915804811194CF0E94011020915904D8
:1045C00030915A042115310509F48ACF10E041E0F9
:1045D00050E0812F90E07A01012E02C0EE0CFF1C0A
:1045E0000A94E2F7B70162237323672B11F41F5F6C
:1045F000F0CF2091570420FF94C0912F990F990F6D
:10460000990F37E0390F80E023E0909313018093F6
:104610001601309314012093170124E630E047E09F
:1046200050E061E171E088E732D5892B09F058CF7D
:10463000B0E21B9FA00111248091570480FF7DC030
:10464000E7E3F2E080E2DF011D928A95E9F760E797
:10465000262E61E0362E0CE611E077E0972E8824B6
:104660008394F10161911F01D8018D918D01840F17
:10467000952F911DFC01E95AFD4F2F01E62FF0E027
:10468000E95CFD4F20E030E0692C621AC82C022E54
:1046900001C0CC0C0A94EAF7520190E0D5018D914B
:1046A0005D018C21662D691B677070E0B82F062EA6
:1046B00001C0BB0F0A94EAF77195619571096770A3
:1046C000772701C086956A95EAF78B2B6081682B66
:1046D00060839F5F983011F72F5F3F4F31962830EE
:1046E000310591F6E4E72E16E1E03E0609F0B9CF78
:1046F00004E610E020E230E047E352E060E488E7BF
:104700005AD5892B09F0ECCEE094F09480915904AD
:1047100090915A048E219F2190935A0480935904BA
:10472000DFCE9695879596958795282F912F929510
:10473000990F90763FE1390F68CF495A5D4F04E6F3
:1047400010E020E230E0DACF00E210E09E012F5FBF
:104750003F4F79018091E80085FD0AC08091E80013
:104760008B778093E8000E94670A811599F3F4CE55
:104770008091F100D7018D937D010150104051F7D8
:10478000EBCEE43148F4E11551F0E150E33138F477
:10479000F0E0E353F44D5AC7EE3F09F4F9CE8FEF42
:1047A000898312C01A8289E08B830EC08A8182308D
:1047B00081F08330B1F0813091F70E94B8094CD775
:1047C0006B837C838D839E83CE0101960E94B70A02
:1047D00096CD88E290E06DD71B821C821D828E836D
:1047E000F3CF8091720490917304892B69F38AE06E
:1047F000E8E6F4E0DE01139601900D928A95E1F768
:10480000E3CF8A81823059F66B817C818D819E81D4
:1048100023D788E290E069D7D7CF4C816B818A811A
:104820000E94370E9827892798279E838D83CCCFA7
:104830002D813E813227232732274C816B818A814B
:104840000E949E0BC1CF0E94C50BBECF80E18A8320
:10485000BBCF81E08A8387EAA7CF8C818D3108F0B6
:10486000B3CF8A809B80982489249824A12CB12CD2
:104870008E010F5F1F4F7801E80EF11C0E151F050A
:1048800009F4A2CF80E0B7EA8B16B1E09B06A10441
:10489000B10420F4C401875A9D4F0BD7F8018483DB
:1048A0000F5F1F4FFFEF8F1A9F0AAF0ABF0AE6CFB5
:1048B0008091720490917304892B09F485CF8C81C7
:1048C0008D3108F081CF882E912CA12CB12CCA807B
:1048D000DB80DC24CD24DC24E12CF12C8E010F5F65
:1048E0001F4F412C512C3201481459046A047B0497
:1048F00008F06ACF27EAC21621E0D206E104F104EB
:1049000038F4D80114966C91C601875A9D4FEDD6A4
:10491000BFEF4B1A5B0A6B0A7B0AEFEFCE1ADE0A77
:10492000EE0AFE0A0F5F1F4FDFCF0E9423104CCF0D
:1049300084E08DCF8C818D3108F046CF882E912C6C
:10494000A12CB12CCA80DB80DC24CD24DC24E12C1A
:10495000F12C412C512C32018E010B5F1F4F48145A
:1049600059046A047B0408F02FCF80E0F0E3CF16EF
:10497000F2E0DF06E104F10418F4C601899699D645
:10498000D8018D938D01BFEF4B1A5B0A6B0A7B0A2E
:10499000EFEFCE1ADE0AEE0AFE0AE1CF2C81022FDB
:1049A00010E02D3108F010CF8A819B81982789274C
:1049B00098272C01612C712C8033F2E09F0708F0BE
:1049C00003CF822E912CA12CB12C40E352E060E069
:1049D00070E04419550966097709421751056105C8
:1049E000710508F4F1CE2091720430917304232BE9
:1049F00009F03EC01C0129E2220E311C80FBEE248E
:104A0000FF24E0F880FF0BC0889653D69D8189274C
:104A10009827892781159C4711F48FEF8D83D50145
:104A2000C401840D951DA61DB71D80FF19C0680126
:104A300081E0C81AD108DE011596AC0DBD1DBAA7DC
:104A4000A9A7C101800F911F34D6E9A5FAA59081CD
:104A500081159C4721F48FEFA9A5BAA58C938601F7
:104A6000FE013196EE0DFF1D2FEFE016F10638F036
:104A70008E010F5F1F4FC12CD12C760125C0948170
:104A8000858181159C4711F42483258332E0E30E50
:104A9000F11C3296EACF80E3481682E058066104A2
:104AA000710430F4D80114966C91C20189961DD618
:104AB000BFEFCB1ADB0AEB0AFB0AEFEF4E1A5E0AD6
:104AC0006E0A7E0A0F5F1F4FC814D904EA04FB0464
:104AD00010F37ACE8091720490917304892B09F4BB
:104AE00073CECE0101960E94B70AFFEF21EE34E0AB
:104AF000F15020403040E1F700C000009ECB88E03C
:104B0000E8E4F1E0DE01919601900D928A95E1F7DB
:104B1000FE0132968FE1DF011D928A95E9F786E06A
:104B2000898388E07F96DE01159666CE8CE58983C1
:104B300081E08A831B821C8247CE0B811C81012E5F
:104B4000000C220B330B45E0000F111F221F331FF7
:104B50004A95D1F7B901A801405E5F4F6F4F7F4F73
:104B6000401751076207730708F42ECE0C35B1E0E9
:104B70001B072105310508F027CE4D35E1E05E0722
:104B80006105710520F04CE551E060E070E0401BEC
:104B9000510BB8016555754F66D516CE4AE150E008
:104BA0006FEF70E0CE0107967DD580917204898306
:104BB0000A8384E08B838C8399E09D8310CE81E00F
:104BC00090E09093A4048093A30482E390E09093F8
:104BD0006704809366040E94AA10909365048093F2
:104BE0006404F2CD0115110581F1D0906C04C090E0
:104BF0007104E0906404F09065040E94AA108E197C
:104C00009F098536910540F1C4FE26C0D4FE24C01C
:104C10000E94AA10909365048093640480916604B6
:104C20009091670401979093670480936604892BA1
:104C300061F41092A4041092A30481E090E0909398
:104C400073048093720400E010E080917204898301
:104C50000A8380916604A8CD82E390E09093670474
:104C600080936604F2CF1092730410927204ACCD5C
:104C700040E250E06FEF70E015D5A6CD2B812111F9
:104C8000A3CD2FE1DC011D922A95E9F781E088A3ED
:104C90009BCD80912802811509F4BBCBB0E1B9BD51
:104CA000E2E1E9BD09B400FEFDCF8091D8008F7D1F
:104CB0008093D8008091E00082608093E000809132
:104CC000E00081FDFCCF0E940511A3CB78941F92D8
:104CD0001FB61F9211248F939F93AF93BF93809120
:104CE000120290911302A0911402B0911502019644
:104CF000A11DB11D8093120290931302A093140280
:104D0000B0931502BF91AF919F918F911F901FBEDD
:104D10001F9018951F920F920FB60F9211242F9388
:104D20003F934F935F936F937F938F939F93AF9333
:104D3000BF93EF93FF938091E10082FF09C08091C0
:104D4000E20082FF05C08091E1008B7F8093E1004B
:104D50008091DA0080FF24C08091D80080FF20C0BD
:104D60008091DA008E7F8093DA008091D90080FFF5
:104D7000A9C080E189BD82E189BD09B400FEFDCFF3
:104D800081E08093740480910102811109C00E9426
:104D9000980A0E941A0B8091E20084608093E200DE
:104DA0008091E10080FF1AC08091E20080FF16C070
:104DB0008091E2008E7F8093E2008091E20080612A
:104DC0008093E2008091D80080628093D80019BC63
:104DD00085E08093740483E0809303018091E10077
:104DE00084FF2FC08091E20084FF2BC080E189BD49
:104DF00082E189BD09B400FEFDCF8091D8008F7D8E
:104E00008093D8008091E1008F7E8093E1008091B3
:104E1000E2008F7E8093E2008091E20081608093C7
:104E2000E20080910002811509F452C084E0809371
:104E3000740480917404843009F052C082E080933D
:104E400003018091E10083FF2CC08091E20083FF89
:104E500028C08091E100877F8093E10082E0809309
:104E60007404109200028091E1008E7F8093E10033
:104E70008091E2008E7F8093E2008091E200806169
:104E80008093E20042E060E080E00E94EA0A8091C4
:104E9000F00088608093F00081E0809303018093AC
:104EA0000201FF91EF91BF91AF919F918F917F91FF
:104EB0006F915F914F913F912F910F900FBE0F9087
:104EC0001F90189519BC109274041092010268CFBB
:104ED0008091E30087FF02C083E0A9CF81E0A7CFE4
:104EE00081E0ADCF1F920F920FB60F921124EF9277
:104EF000FF920F931F932F933F934F935F936F9363
:104F00007F938F939F93AF93BF93CF93EF93FF9331
:104F100009EE10E0F8018081C091EC008F70C79518
:104F2000CC27C795C82B108280EFE82EF12CF70113
:104F30008081877F808378940E942C11F8011082F1
:104F4000F701808188608083CF70F801C083FF9172
:104F5000EF91CF91BF91AF919F918F917F916F9181
:104F60005F914F913F912F911F910F91FF90EF9083
:104F70000F900FBE0F901F901895FF920F931F93E5
:104F8000CF93DF93182FEB011092BC0084EA80933B
:104F9000BC000E94AA10082FF92E8091BC0087FF48
:104FA00028C08091B900887F883029F08091B900AD
:104FB000887F803199F51093BB0084E88093BC0012
:104FC0000E94AA10182F092F8091BC0087FF1EC0D5
:104FD0002091B900287F80E090E0283199F081E0AD
:104FE00090E0203411F480E090E091958195910952
:104FF00009C0802F9F2D0E94B115C817D90768F6E8
:105000008EEF9FEFCDB7DEB7E5E006C3812F902F7F
:105010000E94B115C817D907B8F6F2CF8FEF9FEFEE
:10502000F1CF1092B9008CE08093B80008950F93EF
:105030001F93CF93DF93EB018093BB0084E88093B1
:10504000BC000E94AA10182F092F8091BC0087FF76
:1050500011C02091B900287F81E090E0283211F43E
:1050600080E090E0919581959109DF91CF911F911A
:105070000F910895CF3FDC0741F3812F902F0E94BD
:10508000B115C817D90708F78EEF9FEFEECFA0E054
:10509000B0E0ECE4F8E29CC2782EB62EA72E6A01AE
:1050A00089010E94AA104C010431110508F10F3F3B
:1050B000100711F1C80164E170E071D2F62EE72EFD
:1050C0006F2D7E2D872D59DFEC01892BC1F4EB2C40
:1050D000FA2CCE0CDF1CEC14FD0411F02097C9F063
:1050E00084E98093BC00CE01CDB7DEB7EDE08CC281
:1050F000FF24F394E12CE4CF85E0F82EFBCF0F3FA3
:105100001007F1F2C4010E94B11508171907C0F683
:10511000DECFB801F70181917F0189DFEC01DBCFA0
:10512000A0E0B0E0E5E9F8E253C2782EB62EA72E53
:105130006A0189010E94AA104C010431110508F18D
:105140000F3F100711F1C80164E170E028D2F62E7C
:10515000E72E6F2D7E2D872D10DFEC01892BC1F4FA
:10516000EB2CFA2CCE0CDF1CEC14FD0411F0209774
:10517000C9F084E98093BC00CE01CDB7DEB7EDE085
:1051800043C2FF24F394E12CE4CF85E0F82EFBCF5B
:105190000F3F1007F1F2C4010E94B115081719075B
:1051A000C0F6DECFF7018491B80141DFEC01FFEFDB
:1051B000EF1AFF0AD9CFA0E0B0E0E0EEF8E207C2B4
:1051C000682E962E5A01690178010E94AA10782E45
:1051D000892E0431110518F10F3F100719F1C8018C
:1051E00064E170E0DCD1162F072F612F702F862D20
:1051F000C4DEEC01892BC1F0FFEFEF16FF06A9F327
:10520000872D982D0E94B115E816F90670F784E9EC
:105210008093BC00CE01CDB7DEB7EEE0F4C111E063
:1052200000E0E3CF15E0FCCFB701892D00DFEC01F2
:105230008501CA0CDB1C0C151D0549F3209739F7B5
:10524000B701F80181918F01F2DEEC01F4CF8EE11C
:105250004A9B02C08A95E1F74A9BFECF08955A986F
:1052600080E28A95F1F75A9A0895FC013BE03A955D
:10527000F1F798E020E080E031E040E14A95F1F775
:10528000880F4A9B02C08160232742E04A95F1F7CC
:10529000000040E14A95F1F79A9579F790E19A95E7
:1052A000F1F799B132E03A95F1F7000040E14A9503
:1052B000F1F792FB992790F992272081920F908322
:1052C0000895A1E0B0E0E6E6F9E289C119828C0117
:1052D0007C01E60EF11CBBDFCE010196C6DFF801B2
:1052E00081938F01EE15FF05B1F781E0998191114E
:1052F00080E02196E6E08FC1529A5A9A089552981A
:105300005A9AEA9AE9E6F0E080818F7C80830895DA
:105310006150770B91E001C0990F6A95EAF7692F08
:1053200090E021E0611108C0911599F05A9A80E24D
:105330008A95F1F75A980895362F3823311539F0A8
:105340005A9A922730E23A95F1F76695EBCF5A9840
:10535000F9CF5A98ECCFFF920F931F93CF93DF931F
:10536000EC018C01060F111DF99079DF68E08F2D9B
:10537000CFDFC017D107C1F7CDB7DEB7E5E04CC12D
:105380001F920F920FB60F9211240F931F932F931A
:105390003F934F935F936F937F938F939F93AF93BD
:1053A000BF93EF93FF93CF93DF930F92CDB7DEB709
:1053B00019824DDFCE01019658DF082F069506951C
:1053C0000695982F92959570202F2570920F292F72
:1053D000237096959695920F982797708981892BBF
:1053E000811509F058C0073008F055C080E18A9552
:1053F000F1F75A9A529A82E08A95F1F700C05A98CA
:1054000088E0089F80011124D801A85EBE4F16963F
:10541000ED91FC9117973097A9F06091740170910C
:10542000750114962D913C911597260F371F1196F3
:105430008D919C911297680F791F13964C91139739
:105440008C910995F801E85EFE4F6381611549F082
:10545000209174013091750184819581820F931F91
:105460007ADFFDDE80E18A95F1F75A9852985A9AD0
:1054700080E18A95F1F7F801E85EFE4F60816115E1
:1054800049F0209174013091750181819281820FE0
:10549000931F17DFDCDE0F90DF91CF91FF91EF912B
:1054A000BF91AF919F918F917F916F915F914F913C
:1054B0003F912F911F910F910F900FBE0F901F9052
:1054C00018950F931F93CF93DF938C0107970CF0E0
:1054D0005EC0F894529A5A9885E08A95F1F70000D8
:1054E000C02FC695C570802F8570C80F8C2F837014
:1054F000C695C69593E0000F111F9A95E1F7C80F66
:10550000C8018C2BEC01ABDE00C068E08C2F00DF03
:1055100090E19A95F1F752985A9A4A9B31C087E0E8
:1055200090E04A992FC0F801E85EFE4F6381611553
:1055300059F0209174013091750184819581820F19
:10554000931FBFDE811501F182DE80E28A95F1F7BB
:105550005A98529A90E19A95F1F7F801E85EFE4F59
:105560006081611549F0209174013091750181814C
:105570009281820F931FEFDE72DE789481E008C083
:1055800000C0CBCF019749F4529A5A9A789480E0A0
:10559000DF91CF911F910F91089500C0C2CFAA1B38
:1055A000BB1B51E107C0AA1FBB1FA617B70710F00E
:1055B000A61BB70B881F991F5A95A9F78095909540
:1055C000BC01CD0108952F923F924F925F926F924E
:1055D0007F928F929F92AF92BF92CF92DF92EF9283
:1055E000FF920F931F93CF93DF93CDB7DEB7CA1B04
:1055F000DB0B0FB6F894DEBF0FBECDBF09942A882F
:10560000398848885F846E847D848C849B84AA84D6
:10561000B984C884DF80EE80FD800C811B81AA8163
:10562000B981CE0FD11D0FB6F894DEBF0FBECDBF2E
:10563000ED010895992778E0880F991F961708F0D3
:10564000961B881F7A95C9F780950895EE0FFF1F66
:105650000590F491E02D099469279627692778270A
:10566000872778270895FB01DC0102C005900D9281
:1056700041505040D8F70895FB01DC0104C08D91E2
:105680000190801921F441505040C8F7881B990BB4
:105690000895FB01DC0102C001900D924150504081
:1056A000D8F70895DC0101C06D9341505040E0F7F8
:1056B0000895F999FECF92BD81BDF89A992780B5DA
:1056C0000895A8E1B0E042E050E02FC0DC01A40F53
:1056D000B51F4150504040F0CB01840F951F2E91D3
:1056E00005D041505040D8F70895262FF999FECFA4
:1056F00092BD81BDF89A019700B4021639F01FBA25
:1057000020BD0FB6F894FA9AF99A0FBE0895039641
:10571000272FECDFEADF252FE9DF242FE7CF0196E3
:10572000272FE4DFE2CFDC01CB01FC01F999FECFAA
:1057300006C0F2BDE1BDF89A319600B40D92415019
:105740005040B8F70895F894FFCF09122F12351280
:105750002F1235128812AA123512B113BE13501629
:105760006C1673167A169116A4163016B016C91652
:1057700002190619F918FE180A190E1912197F25AF
:1057800096259D25E423E423CE25DF25F225332627
:105790003826E423E423E4233E26D223D62301241F
:1057A0000D2418242324CF23CF23CF23CF236A25EE
:1057B000262429242D245824952498249A24CE2460
:1057C0000000010001B509510CED09EE09670C4814
:1057D0000C0021007F2200030000000100000000F7
:1057E00000000005010000000406000000000000A9
:1057F000010A000000000000010B00000000000092
:10580000010C000000000000E4993598BCC5A0110F
:10581000004422320001DE00AC004A076307830720
:10582000946697C634F4F5F6F73133320008101851
:10583000181008008504E200E900EA00B500B6008F
:10584000B700CD008301CC008A01920194012102AE
:10585000230224022502260227022A02B300B400F2
:105860006F0070009F01CB019F02A002E200E900DF
:10587000EA00B500B600B700CD008301CC008A0174
:10588000920194012102230224022502260227020A
:105890002A02B300B4006F0070009F01CB019F0289
:0258A000A00264
:00000001FF
